:020000001028C6
:080008008B139200030E91001E
:1000100009280000110E8300920E120E8B170900A2
:10002000831609308500FF30860083128501860122
:10003000861838281B28C6202708A71B252827082C
:1000400097001608B7207E201B281F302705960032
:100050001B2849201D089D171D08EF201E08EF20B2
:10006000B720292811309600003097007E203728CD
:100070004920B9201D08031D3828103096001E089D
:100080009700113C03194728013C031D38287E20A6
:1000900038280511051C4928BB209B019C010D3007
:1000A0009A00BD209B0D9C0D1B10051C1B146D2080
:1000B000BB20BD209A0B52281B089E001E139E13C6
:1000C0009B0D9C0D9B0D9C0D1C089D009D131D13ED
:1000D0009D121C1F1E171E080800093098002030B2
:1000E0009900990B7128051878281B1C08007A289C
:1000F0001B180800980B6F280515080083208A201C
:10010000902099200800AB20171B8828AB200800FE
:10011000AE200800930A131CAB201318AE20080071
:100120000530950016089400940D940D940DA120AF
:1001300008000630950017089400940D940DA12036
:100140000800940D0318A628AE20A728AB20950B15
:10015000A12885100800B420B1200800B120B420E7
:1001600008008514BD2008008510BD2008002D3032
:10017000BE28FF30BE280930BE28123098000F304C
:100180009900990BC128980BBF280800A8010830D6
:100190009800851DC628EA20851DC628E2208519FD
:1001A0000310851D0314A80C980BCE28E220851996
:1001B000C628E2208519C6282808A70008000F30A5
:1001C0009900E4280F309900000000000000990B0E
:1001D000E42808000F309000900BEC280800A800DD
:1001E000083098000511DF200515DF20A80C031842
:1001F0000511031C0515DF20980BF6280511DF20DB
:100200000800FA309F00052108006E30A0000000B1
:1002100000000000000000000000A00B07299F0B59
:040220000529003478
:00000001FF
